:020000040000FA
:02000000602876
:080008008610241C8614C000C0
:10001000030EC10083120513251B2428861F1628F2
:100020002208A400241C86142418861006181628FA
:100030000F30A9008B100314061F0310A40C410EEF
:100040008300C00E400E0900861B2C282208A40045
:10005000241C861424188610061C2C280F30A90096
:100060008B100314061B0310A40C410E8300C00E5A
:04007000400E090035
:1000C000A001A101A201A401A501AA01A601A70105
:1000D000A801A80AA901B101B201B301B401B50197
:1000E000B601B701B801C001C1018316FF30850018
:1000F000860086108312851B2514851F2510831604
:1001000085138312AA102A10051F2A14051BAA148E
:100110002A1C8D288316051383128501860107305A
:100120009F00C7308316810083127E3092007D309D
:10013000831692008312003083168C008312903055
:100140008B00A20BA1288B138316011383128B172C
:1001500064000B19D620B5202518B028061EA82843
:100160002A18E320AA189421A82825170800A9080E
:1001700003190800A803031D08001E30A800861FED
:10018000CE28A60A031D08002517A517A601A7015A
:100190008B138316011383128B170800A70A031D04
:1001A00008002513A517A601A70108000B11A9082F
:1001B0000319DF288513251C8517A90308000509E5
:1001C0008039850008008C1C08008C100517000081
:1001D000000000000000000000000000000000001F
:1001E0000000000000000000000000000508A00062
:1001F0000608A1000513201902299630B102031C3C
:100200000B290E299630B107031807290E29FF3054
:10021000B10022140E29B10122100E29A0191529AE
:100220009630B202031C1E2921299630B20703180A
:100230001A292129FF30B200A2142129B201A210EB
:100240002129211928299630B302031C3129342988
:100250009630B30703182D293429FF30B300221537
:100260003429B30122113429A1193B299630B40253
:10027000031C442947299630B4070318402947290D
:10028000FF30B400A2154729B401A2114729A018D4
:100290004E299630B502031C57295A299630B507C6
:1002A000031853295A29FF30B50022165A29B501DF
:1002B00022125A29201861299630B602031C6A2995
:1002C0006D299630B607031866296D29FF30B600F0
:1002D000A2166D29B601A2126D29A11A74299630B1
:1002E000B702031C7D2980299630B70703187929A6
:1002F0008029FF30B70022178029B70122138029F7
:10030000211A87299630B802031C90299329963028
:10031000B80703188C299329FF30B800A217932936
:10032000B801A213932908008C100508A000060844
:10033000A100201AA0290130B1070318A529AC2972
:100340000130B102031CA929AC29FF30B1002214ED
:10035000AC29B1012210AC29A11AB3290130B2078E
:100360000318B829BF290130B202031CBC29BF29D8
:10037000FF30B200A214BF29B201A210BF29A119F7
:10038000C6290130B3070318CB29D2290130B302A3
:10039000031CCF29D229FF30B3002215D229B30183
:1003A0002211D2292119D9290130B4070318DE29D5
:1003B000E5290130B402031CE229E529FF30B4002D
:1003C000A215E529B401A211E529A019EC290130F3
:1003D000B5070318F129F8290130B502031CF529E6
:1003E000F829FF30B5002216F829B5012212F829A4
:1003F0002019FF290130B6070318042A0B2A0130FF
:10040000B602031C082A0B2AFF30B600A2160B2ADC
:10041000B601A2120B2A2018122A0130B7070318BE
:10042000172A1E2A0130B702031C1B2A1E2AFF307E
:10043000B70022171E2AB70122131E2AA018252A48
:100440000130B80703182A2A312A0130B802031CE8
:100450002E2A312AFF30B800A217312AB801A21380
:04046000312A080035
:084000000F00040001000000A4
:02400E00543F1D
:00000001FF
